S31508001800080A0020D9180008E7180008E91800088F
S3150800181000000000000000000000000000000000BA
S315080018200000000000000000000000000119000888
S31508001830000000000000000003190008A93A00088B
S315080018404D49000807190008071900080719000874
S31508001850071900080719000807190008012A0008CF
S31508001860071900089D270008071900080719000826
S31508001870071900080719000807190008153D000888
S31508001880693D000800000000000000000719000874
S3150800189000000000071900080719000807190008C2
S315080018A0000000000719000807190008ED400008A5
S315080018B007190008071900080719000800000000A2
S315080018C0EE11AA550348854600F0D6FB00480047A6
S315080018D0D1680008080A00200B4880F308880B48DE
S315080018E080470B480047FEE704207146084202D0AD
S315080018F0EFF3098001E0EFF30880714604F0CCFDB0
S31508001900FEE7FEE7FEE7FEE7080A0020A93C000816
S31508001910C518000830B50B460146002020220124D0
S3150800192009E00D46D5409D4205D31D469540491B05
S315080019302546954040191546521E002DF1DC30BD4E
S3150800194070B500242546002801DA01244042002902
S3150800195001DA01254942FFF7DDFFAC4200D04042DB
S31508001960002C00D0494270BD03460B439B0703D0A9
S3150800197009E008C9121F08C0042AFAD203E00B7846
S315080019800370401C491C521EF9D27047D2B201E0BE
S315080019900270401C491EFBD270470022F6E710B5BC
S315080019A013460A4604461946FFF7F0FF204610BDBF
S315080019B0F8B502464A40D40F42004B0052085B086D
S315080019C09A4202D20246084611464A0023D0C30D5F
S315080019D04A00DDB2120EAD1A202D35DA490201266B
S315080019E0490AF6058A19002C00D0524220214F1BBD
S315080019F01146B9402A411018C20D9A4221D0002C2E
S31508001A0017D0012D08DCDA05801AD20F8019D20703
S31508001A10DBB200F045F9F8BDDA05801A012340006B
S31508001A201B06C01880185A428018CA0F104349006E
S31508001A3007E04908C2071143DA05801A80194008E9
S31508001A40801800F025F9F8BD61000122511A001B23
S31508001A50F7E70122D2075140AAE70122D2075040F0
S31508001A60A6E7024670B54A40D30FDB0740002DD0E3
S31508001A704A002AD0010E140E000212020919400A61
S31508001A80520A8418E50104465443000A120A2E0431
S31508001A905043A4194219200CC543AA18120C012553
S31508001AA0AD03521C521912047F39240400D0521C6B
S31508001AB0104301D44000491EC2B20C06C0092018C2
S31508001AC0401C4008802A02D003E0002070BD400870
S31508001AD04000002900DA0020184370BD70B50246A0
S31508001AE04A40D50F40004A00ED0740085208002832
S31508001AF014D0002A12D0C40DD30D41020120C0050E
S31508001B005202490A520AE41A091812187D349142F7
S31508001B1001D3641C00E04900002C01DA002070BDE6
S31508001B200023914201D3891A03434008490000283B
S31508001B30F7D100290AD0914202D10121C90705E04F
S31508001B40914201D2012101E00121C943E005C018F3
S31508001B50401900F09DF870BD10B500229623114675
S31508001B6000F09EF810BD410040020122400AD2054D
S31508001B70090E80187F2901DA00207047962903DCB0
S31508001B809622511AC8407047963988407047C20F46
S31508001B90D207400040080BD0C10D0723DB01C91846
S31508001BA040020905400A1143C2084007114370471D
S31508001BB0002001467047000010B5002904DB012407
S31508001BC0E40740428C412146002B04DB1C460123D6
S31508001BD0DB075242A3418B4200D1824210BD00006E
S31508001BE010B5002904DB0124E40740428C41214654
S31508001BF0002B04DB1C460123DB075242A341994212
S31508001C0000D1904210BD00000122D207002800DB57
S31508001C10101A002900DB511A814270470122D207A7
S31508001C20002800DB101A002900DB511A8842704789
S31508001C30F0B51FB40646002082B00546402401913F
S31508001C4000901BE0019922460F46304600F036FA0E
S31508001C50049A059B801A994110D3104619462246C4
S31508001C6000F01CFA361A8F410197224601200021FE
S31508001C70009F00F013FA38184D4100902046641E64
S31508001C800028DFDC019B00982946324607B0F0BDE4
S31508001C90002904DA401C490001D140084000704779
S31508001CA070B40024050C05D11024000402D10029C3
S31508001CB021D01124050E01D100020834050F01D1E7
S31508001CC00001241D850F01D18000A41C002801DB1A
S31508001CD04000641C002908D020252E1B0D46F5401F
S31508001CE0A14000D001212943084301061B1B000A15
S31508001CF0DB1D02D5002070BC7047DB05181880185C
S31508001D000029F8DA401C4900F5D170BC40084000AB
S31508001D1070470000F0B507460846584087B0C00F20
S31508001D20049048000E46590040084908BC1A8841E4
S31508001D3005D2384631461E4617460B460246580017
S31508001D40400810434CD0300D039040055900400D13
S31508001D50490D0590401A0290402872DA18030121AD
S31508001D60000B09050843019004980092002805D045
S31508001D700199524200208841009201900298402120
S31508001D800A1A0199009800F089F905460C466B462F
S31508001D9007CB00F0A4F9C0197141039A0E0D002370
S31508001DA0D71756401A467A40164344D0049A002A52
S31508001DB02DD0029A012A039A15DC1205C01A914100
S31508001DC001263605001C7141D20F059ED2070093E5
S31508001DD0019202962A46234600F0A1F907B0F0BD03
S31508001DE038463146FAE71605224A0F46B218C01A8F
S31508001DF0B74101210905001C4F4100187F411146D2
S31508001E0018187941E20F10436D19644113E0E2078F
S31508001E106D0815436408C2071443039A0126120580
S31508001E20C01A91413605001C7141CE07400830435F
S31508001E304908C01851412A46234600F063F9CDE700
S31508001E40FFE7049801224000C117121A00238B41AC
S31508001E5004983146C417381AA141EEE730B4012474
S31508001E60E407634030BC55E730B40124E407614019
S31508001E7030BC4FE70000E0FFF0B51FB488B00B99FF
S31508001E800998002448400999C00F49004908099152
S31508001E90C0070B990090490049080B9109990898C1
S31508001EA0A64608431CD00B990A98084318D00998E7
S31508001EB001244000420D4800410D099824050003FD
S31508001EC0000B204309900B980003000B20430B904E
S31508001ED050181C494018002201901446104605E087
S31508001EE0002001460DB0F0BD032801DA034600E0E4
S31508001EF003239C46C11A0AAE0AE05F0008ADED5BF3
S31508001F004F00F75B7D430027AA187C41491C5B1EDE
S31508001F106145F2DD410004AB5A522104120C0A4312
S31508001F20240C401C0828DFDB0198029000997046B3
S31508001F3001910090059B049A0799069800F0EFF81E
S31508001F40D0E700000DFCFFFFF0B50C465C4085B0FD
S31508001F50E40FE40703944C000026640859009446ED
S31508001F60490802460296224321D062460A431ED0F9
S31508001F706200570D4A000E032303550D012402463D
S31508001F802C492405781B1B0B360B40182343264384
S31508001F90614600901C46501AB44103D30098401C71
S31508001FA0009002E0921800985B41002803DA0020AE
S31508001FB0014605B0F0BD0020012109050746864601
S31508001FC011E064461D46141BB54106D36546521BEF
S31508001FD0B341744607430C43A646CD074008490853
S31508001FE0284392185B4105460D43EAD1104618432B
S31508001FF013D06046194650407140084306D06046E3
S31508002000101AB34106D20122002306E0002201235A
S31508002010DB0702E00122D2435310009874460105FB
S31508002020381C6141029C039D0019694100F06AF859
S31508002030BFE70000FD0300004A0009030123090B5E
S315080020401B0519430A4B10B5520D9A4202DA0020B5
S31508002050014610BD064B34339A4203DC9A1A00F047
S315080020602DF810BD034BD21800F018F810BD00006B
S31508002070FF030000CDFBFFFF064C0125064E05E0D9
S31508002080E36807CC2B430C3C98471034B442F7D38B
S31508002090FFF71CFC187600083876000810B5202AC9
S315080020A004DB0146203A9140002010BD91402023D0
S315080020B09C1A0346E3401943904010BD10B5202AE8
S315080020C004DB0846203AD040002110BD0B46D34019
S315080020D0D0402024A21A91400843194610BD10B5D5
S315080020E0202A06DBCB170846203A1041C1170B43B6
S315080020F006E00B461341D0402024A21A914008431B
S31508002100194610BD10B5002B08DA0024401C6141A1
S3150800211092185B411A4301D14008400010BDF0B542
S315080021201FB482B005460C0003D0084602F07AFCBC
S3150800213002E002F077FC203002460090214628464D
S31508002140FFF7ACFF049B059A04460F461843114354
S31508002150084314D0184610431BD0009840210A1A89
S3150800216018460599FFF7AAFF05460E46009A0599EF
S315080021700498FFF793FF084305D0012004E02046A2
S31508002180394607B0F0BD0020C11705430E432C435E
S31508002190374300990E986305401A7905E40A002228
S315080021A00C43FD0A0A3002D500200146E9E701057D
S315080021B0101969410C9C0D9D00196941FFF7A2FF92
S315080021C0DFE7000010B50446002C08D101210920DC
S315080021D0C00600F0B5FE002000F0AAF852E0012C77
S315080021E005D102210920C00600F0AAFE4AE0022C09
S315080021F005D104210920C00600F0A2FE42E0032C06
S3150800220005D108210920C00600F09AFE3AE0042C00
S3150800221005D110210920C00600F092FE32E0052CF7
S3150800222005D120210920C00600F08AFE2AE0062CE6
S3150800223005D140210920C00600F082FE22E0072CC5
S3150800224005D180210920C00600F07AFE1AE0082C84
S3150800225004D101210D4800F073FE13E0092C04D1C6
S3150800226002210A4800F06CFE0CE00B2C04D1102168
S31508002270064800F065FE05E00C2C03D180210348D2
S3150800228000F05EFE204600F053F810BD000400483A
S315080022907FB50020009001900290039000241BE077
S315080022A000250CE0E8000E4940186100405AA100DC
S315080022B06A4651584018A1005050681C85B2142D22
S315080022C0F0DBA1006A4650581421FFF723FB610092
S315080022D0044A5052601C84B2042CE1DB7FBD000026
S315080022E0600400204C01002000B587B001A800F06A
S315080022F0AFF80121480201F049FA00200190302088
S31508002300029001204002039000200690059001A942
S31508002310064800F031F80121044800F021F80121AF
S31508002320024800F011F807B000BD00000024014083
S3150800233010B50446072300222146024800F038F863
S3150800234010BD000000240140002904D04268012382
S315080023501A43426003E042685208520042607047DE
S31508002360002904D0826808231A43826003E0826841
S3150800237008239A438260704742680B4B1A404260B2
S315080023800B684A681A4343681A4342608268074BD7
S315080023901A4082600B694A691A438B681A43836834
S315080023A01A438260704700000FBCFFFF8FF1F9FFE8
S315080023B0F0B504460D4616461F463F073F0F2B4607
S315080023C0082B0FD91B071B0F083B606F9A000F21BC
S315080023D0914088436067606F99003A468A40104387
S315080023E060670BE0206F9A000F21914088432067B1
S315080023F0206F99003A468A4010432067E068012119
S31508002400A9408843E060E0680121A9400843E060EC
S31508002410012080032840002803D0012000F020F87E
S3150800242007E00120C0032840002802D0012000F060
S3150800243017F8F0BD002905D08268FF2301331A4337
S31508002440826004E08268FF2301339A438260704702
S31508002450002101604160816001730161416170473B
S31508002460002806D0064949680C221143044A5160DF
S3150800247005E0034949680C229143014A51607047B7
S315080024800024014010B507480078002806D0FFF759
S31508002490FFFE00200349087000F09CFD7E2002F034
S315080024A061FA10BD54010020FFB583B00C460294B2
S315080024B000200190002726E000261CE0721C0399E4
S315080024C051430846791CFFF725FA0546A54201D966
S315080024D0281B00E0601B05460298A84204D902950D
S315080024E005980670069807700298002802D1012000
S315080024F0019002E0761C402EE0D300BF0198002828
S3150800250000D002E07F1C042FD6D300BF029807B084
S31508002510F0BD000000BF00BF00BF00BF00BFBFF393
S315080025204F8F00BF00BF00BF06480749C86000BFFD
S3150800253000BF00BFBFF34F8F00BF00BF00BF00BF83
S3150800254000BFFDE70400FA0500ED00E010B500F055
S3150800255001F810BD10B523480078002817D1224885
S3150800256001F09CF901283CD11F480078002838DD85
S315080025701D480078402834DC01F08BFD1B490860B3
S3150800258001201849087000201949087029E0164AE0
S3150800259017490978491C501801F080F9012816D105
S315080025A013480078401C124908700F4800780978CB
S315080025B0884216D100200B4908700B484078FF283E
S315080025C00FD10B48007802280BD1FFF7A3FF01F0C3
S315080025D060FD064909686431884202D9002001492C
S315080025E0087010BD21010020E4030020240100200A
S315080025F02001002078B50246002327E0002020E0CD
S315080026008400155B441CA400145BA54218DD8400F5
S31508002610A5182E886C4626806D8865808400A518C6
S31508002620441CA400A41826882E8064886C80441C48
S31508002630A400A5186C4624882C806C4664886C8097
S31508002640401C4C1EE41A8442DADC5B1C4C1E9C427D
S31508002650D4DC78BD10B586B004460121880301F0A4
S3150800266095F80121880401F071F8032211462248E1
S3150800267000F051FC032204211F4800F04CFC01A87D
S3150800268001F0D9FD0194302168460181002141817C
S31508002690818101821821C18101A9184801F088FDAC
S315080026A00121164801F061FD05A800F08AFC082101
S315080026B068468182012181751821C17505A90E48D0
S315080026C000F0DCFB1021684681824821C17505A906
S315080026D0094800F0D3FB1B216846017003214170AD
S315080026E00121817000F098FF01220221034801F0C0
S315080026F054FD06B010BD0000000400480038014033
S3150800270070B502460B46FF25FF2408E01178521CD7
S3150800271069400748405C604005460648445C1846E0
S315080027205E1EB3B20028F1D12802204370BD000016
S31508002730187400081875000801B50649009808605D
S3150800274002E07E2002F00EF9024800680028F8D15F
S3150800275008BD00002C010020014600220E4B1A611C
S31508002760CA005A6100229A6105221A6100BF0A4A04
S315080027701069C207D20F002A04D0012212040240AF
S31508002780002AF4D0044A126952085200024B1A6110
S3150800279000229A617047000000E000E010B50021B1
S315080027A00848FFF747FE022000F052F801200649C4
S315080027B0087001020920C00600F0FFFB02F0FAFDCE
S315080027C010BD0000002401405C01002000B589B05E
S315080027D00121084600F0BAFF1A4800F045F801A89A
S315080027E000F08EF8184801901848029000216846B3
S315080027F001730420049068460175802141754900DB
S31508002800C182890001832021817609028183002102
S31508002810C183018401A90B4800F04CF8012109483D
S3150800282000F01CF801220221064800F039F80921B7
S3150800283068460170022141700121817000F0ECFEAA
S3150800284009B000BD08000240002401402804002009
S3150800285001494860704700000000024002685208BB
S3150800286052000A430260704710B5044620684008C3
S3150800287040002060002020606060A060E060E1B257
S31508002880084608380521FFF745F801460F20884015
S315080028900249496808430149486010BD00000240E2
S315080028A0002A03D003680B43036002E003688B43E6
S315080028B00360704710B50A7A8B7D1A430B7C1A435E
S315080028C04B7C1A434B8A1A438B8A1A430B8B1A433F
S315080028D04B8B1A430368094C23401A43026002686B
S315080028E00123DB039A438B8B1A430260CA68426052
S315080028F00A6882604A68C26010BD00000F80FFFF48
S315080029000021016041600172C16001744174418215
S3150800291081828175018341838183704770B506463C
S315080029200C4621460A4800F00FFA0546002D01D14B
S31508002930401E70BD0648854202D10648051B00E0C8
S315080029402D1B224629463046FFF70EF82046F0E7AB
S3150800295000F4000800FC000870B506460C4621463F
S315080029600A4800F0F1F90546002D01D1401E70BD58
S315080029700648854202D10648051B00E02D1B224663
S3150800298029463046FEF7F0FF2046F0E700F000083B
S3150800299000F8000870B506460C4621460A4800F0BD
S315080029A0D3F90546002D01D1401E70BD0648854263
S315080029B002D10648051B00E02D1B22462946304653
S315080029C0FEF7D2FF2046F0E700F8000800000108ED
S315080029D070B505460C4622460249284600F075F9A8
S315080029E0204670BD00F4000870B505460C46224620
S315080029F00249284600F069F9204670BD00F0000833
S31508002A0010B5024800F004F810BD00002080000050
S31508002A100149486170470000000401401CB568463A
S31508002A2000F0A9F80F21002000F07CF80120C0036F
S31508002A3000900021684601711021417101218171C0
S31508002A4000F010F80521002000F06CF82020009016
S31508002A50002168460171102141710121817100F040
S31508002A6001F81CBD8179002948D02D4909680268FA
S31508002A7091432B4A11601146496802689143284AD6
S31508002A8051600179002906D1114609680268114387
S31508002A90234A116005E02249496802681143204A21
S31508002AA051601F498968026891431D4A9160114621
S31508002AB0C968026891431A4AD160417910290CD134
S31508002AC01146896802681143154A91601146C9681A
S31508002AD002681143124AD16020E04179082906D1DB
S31508002AE00F498968026811430D4A916016E00C493E
S31508002AF0C968026811430A4AD1600FE001790029C2
S31508002B0006D10749096802689143054A116005E03C
S31508002B100349496802689143014A516070470000B9
S31508002B200004014010B50D4A8B109B00D3588A0744
S31508002B30140F0F22A2409343084A8C10A400135185
S31508002B408B109B00D2588B071C0F0346A3401A43D1
S31508002B50024B8C10A4001A5110BD00000800014059
S31508002B6008B507216846017002214170012181706C
S31508002B7000F052FD08BD0021016001710C21417170
S31508002B80002181717047000010B5044608480069A5
S31508002B900221084306490861084644610069402144
S31508002BA0084303490861034800F00EF910BD000008
S31508002BB000200240FF0F00000C48C068C007C00F85
S31508002BC0002801D0012070470848C0680421084041
S31508002BD0002801D00220F6E70448C0681021084002
S31508002BE0002801D00320EEE70420ECE7002002408D
S31508002BF003480069802108430149086170470000BD
S31508002C000020024030B504460D46054800690121FA
S31508002C1008430349086125800F2000F0D5F830BD28
S31508002C200020024010B57E2001F09CFE064800F008
S31508002C300FF87E2001F096FE044800F009F87E2081
S31508002C4001F090FE10BD000000F4000800F0000836
S31508002C5010B5044600F0ACF82046FFF795FFFFF7DD
S31508002C60C7FF10BD70B503460125002208E05000D5
S31508002C701C5A0748844201D0002506E0501C82B23F
S31508002C80CE0F761876109642F1DC00BF284670BD46
S31508002C90FFFF0000F8B505460E46144600F088F812
S31508002CA07E2001F05FFE002707E029883046FFF7FF
S31508002CB0A9FFB61CAD1C781C87B2E10F091949108B
S31508002CC0B942F2DCFFF794FFF8BDF8B507460C46A3
S31508002CD015462946204600F037F80646002E0DD13F
S31508002CE02046FFF7B5FF012080022018FFF7B0FF46
S31508002CF02A4621463846FFF7CDFF24E00120800208
S31508002D002018401BB0420AD1012080022018FFF784
S31508002D109FFF2A4631463846FFF7BCFF13E00120DD
S31508002D20C0022018401BB04208D12046FFF790FF8A
S31508002D302A4631463846FFF7ADFF04E02A463146B3
S31508002D403846FFF7A7FFF8BDF8B505460E462F46E5
S31508002D50E807C00F002801D000BFFEE73146012072
S31508002D60C002FEF7EDFD002901D000BFFEE70024F2
S31508002D700BE020467043471931463846FFF772FF85
S31508002D80012800D108E0601C84B231460120C00247
S31508002D90FEF7D6FDA042ECDC00BF31460120C0029A
S31508002DA0FEF7CEFDA04200D100273846F8BD000048
S31508002DB0024803494860034848607047230167454D
S31508002DC000200240AB89EFCD10B5024600BFFFF7E1
S31508002DD0F3FE0346521EFF2400E0641E002CFCD1BD
S31508002DE0012B01D1002AF2D10648006977218843D0
S31508002DF0044908613420C860002A01D1052010BDA5
S31508002E001846FCE70020024008B5684600F0D9F8E5
S31508002E1001210F20400400F099FC0021C9436846AF
S31508002E2001800021C17069460920C00600F026F815
S31508002E300021C943684601800021C17069460C48D3
S31508002E4000F01CF80021C943684601800021C170C2
S31508002E506946084800F012F80021C943684601800F
S31508002E600021C1706946044800F008F808BD000052
S31508002E700004004800080048000C0048F8B502465F
S31508002E80CD782F073F0FCD7810263540002D01D07D
S31508002E908D782F431446002011E085062B0E0D88E9
S31508002EA0012686403540002D07D025680F269E400E
S31508002EB0B5433E469E4035432560451CE8B2082882
S31508002EC0EBDB141D0D882D120095002011E08506F8
S31508002ED02B0E01258540009E3540002D07D025681C
S31508002EE00F269E40B5433E469E4035432560451C09
S31508002EF0E8B20828EBDBCD78282D04D155690E8871
S31508002F003543556106E0CD78482D03D115690E88FD
S31508002F1035431561F8BD70B54D07EB0E082902DA81
S31508002F200546203501E0054624352C460F269E40E9
S31508002F302568B54316469E403543256070BD00009A
S31508002F4038B504460D460920C006844203D101213E
S31508002F50480400F0FBFB1148844203D1012100021A
S31508002F6000F0F4FB0E48844203D10121000200F070
S31508002F70EDFB0C48844203D10121080500F0E6FB6D
S31508002F80684600F01EF86846058001218170002118
S31508002F90C17069462046FFF771FF38BD0004004836
S31508002FA000080048000C00480246906808400028BF
S31508002FB001D0012070470020FCE74161704701619C
S31508002FC070470021C9430180022181700421C17024
S31508002FD070470000F0B587B0002006900590049071
S31508002FE003907E2001F0BEFC002611E07100BB4A6A
S31508002FF0505AFEF7B1FD0546B949FEF76FFD04467E
S31508003000B849FEF72EFDB100B74A5050701C86B27B
S31508003010042EEBDBB44A51689068FEF71AFD0446A5
S31508003020B249FEF75BFD0690AF4948680699FEF778
S3150800303055FDAF49086008460068FEF7A8FD044636
S3150800304022460B46ABA001F0DDFCAD48807B00288C
S315080030503FD1AB4910318889FEF77EFDA84910316A
S315080030600190C888FEF778FDA6490090FEF736FD60
S3150800307007460199FEF7F5FC0546A349FEF72EFD1E
S3150800308004469F4910318889FEF766FD07469E4922
S31508003090FEF724FD0546964801682846FEF7DDFC3E
S315080030A021460290FEF71AFD049095491031488989
S315080030B0FEF752FD05460499FEF77AFC0446FEF72C
S315080030C052FD924908600846008881B2904881817D
S315080030D034E08F48007D002830D18948C07801281F
S315080030E029D183480068FEF752FD0446894A8A4B6F
S315080030F0FEF776FD1CD27E480068FEF748FD0446BA
S31508003100864A874BFEF758FD12D27F4978480068F1
S31508003110FEF7A7FC0446FEF726FD81B27848103074
S3150800312081810146888903F033FD03F09DF802E0AA
S31508003130022003F091FD0021714881737048C07B1D
S31508003140012804D103F090F800216D48C173704935
S315080031508889FEF701FD7349086063490868724962
S31508003160FEF77FFC054601218907FEF77AFC04462F
S31508003170FEF7F9FC81B266484181FF38C1380088FC
S31508003180FF21F531884272DD00205D493439088017
S315080031905B48C07801283ED15D48007D00283AD0BA
S315080031A0514988686049FEF75CFC0446FEF7DBFC7B
S315080031B085B24D4948685C49FEF753FC0446FEF75C
S315080031C0D2FC80B2854210D14D483438C068AF2150
S315080031D08900884209D94E484079002805D14849CE
S315080031E03439C86004214A4841713F49886800213A
S315080031F0FEF70AFD05D03C4948680021FEF704FDA4
S3150800320009D143484079002805D13D493439C86079
S3150800321005213F4841713449C868FEF7B8FC0446A1
S31508003220424A434BFEF7C8FC22D22F49C868FEF72C
S31508003230AEFC04463F4A404BFEF7BEFC13D22021A3
S315080032403E48FFF7B1FE00280DD131480079012824
S3150800325009D12F484079002805D129493439C86051
S3150800326006212B48417101212548417011E033E0C0
S315080032701D49C8683249FEF7D1FC0AD22448007DA8
S31508003280002803D100211E48417002E001211C4894
S3150800329041701549C8682B49FEF7C0FC03D20121C5
S315080032A01748017102E00021154801711448407859
S315080032B000280DD116480079012804D104211F4899
S315080032C0FFF77BFE08E004211C48FFF778FE03E0C1
S315080032D004211A48FFF773FE07B0F0BD4C01002021
S315080032E000F07F450000A040500400203333A3407F
S315080032F0600100200A525F313A25660A0000000084
S31508003300000200200024744900007A446801002065
S315080033108C030020666666666666E63FCDCCCCCC36
S31508003320CCCCEC3FA40300200000C842A245B6F36B
S31508003330FDD4EC3F75931804560EDD3F0004004893
S3150800334052B89E3FFCA979400148006870470000C2
S3150800335030010020034800680349097840180149EC
S3150800336008607047300100203801002008B50121A7
S31508003370480400F0EBF90121880400F0E7F96846F3
S31508003380FFF71FFE0421684601804821C17069467F
S315080033900920C006FFF772FD6846FFF712FEFF21F7
S315080033A00131684601804821C17069460748FFF720
S315080033B065FD6846FFF705FE202168460180042161
S315080033C0C17069460148FFF759FD08BD0004004869
S315080033D010B504210920C006FFF7E6FD00286FD1C5
S315080033E05E48407A00285FD15C48007901283DD1C3
S315080033F05A48007D002839D159480078401C584958
S31508003400087008460078042823DB56A001F0FAFA6B
S3150800341000205349087051487C38408900280AD151
S3150800342052485349C860012151483430C172FF30AF
S31508003430113041810AE002214D483430C172002022
S315080034404B49C860002145487C38418101F0AAFAF9
S315080034500CE043480078022808DC4548C0687D210E
S315080034600901884202D900204149C8603B48007DCD
S31508003470002816D13E48C0693E49884211D33748CC
S315080034807C384089002805D13B483949C861002065
S31508003490C86006E032480078022802DC0020344979
S315080034A0C86001212D4841723448007800280ED1A1
S315080034B001203249087001212848017207E0FFE718
S315080034C000202E49087000212448017241722848BC
S315080034D000697D21C90088423AD929A001F092FAEB
S315080034E000202349086100211C480172007D00283C
S315080034F028D11A487C384088032829DA17487C38A6
S315080035004089002824D11A483430007900280ED181
S315080035101248007901281BD10121104801750020A5
S315080035201349C860012112483430C17210E00B48B3
S31508003530407900280CD101210848417100200C4926
S31508003540C86005E000200A49C860002103480171E7
S315080035507E2001F007FA0148007A10BD8C0300208E
S31508003560C40000204C4F434B45442100DC050000B5
S31508003570CC01002030750000606D00007601002047
S315080035800A537461727420576F726B0A0000000048
S315080035901CB50121480400F0D9F80121880400F07F
S315080035A0D5F801A8FFF70DFD442168468180012161
S315080035B081711021C17101A91548FFF75FFC1549F2
S315080035C068468180012181711021C17101A90920F4
S315080035D0C006FFF753FC08210920C006FFF7EFFCD9
S315080035E000BF8021684601800021C1706946092014
S315080035F0C006FFF743FC20210920C006FFF7DFFCC1
S3150800360000BF10210920C006FFF7D9FC1CBD000029
S3150800361000040048798100008178002925D01749DF
S3150800362003221202891802789210920089580278A9
S315080036309207D30EFF229A40914342789207120EC0
S3150800364003789B07DB0E9A4011430C4A03231B029F
S31508003650D21803789B109B00D1500178CA06D20E67
S3150800366001219140054A116007E00178CA06D20E89
S3150800367001219140014A80321160704700E100E063
S3150800368009480A494860002048875A2088870887D9
S31508003690074808630020C8620648486206488862E8
S315080036A00448C8617047000000003443A4030020A2
S315080036B09A99993E00002041000048420D4A126836
S315080036C09208920002430B4B1A600B4A12690423B4
S315080036D01A43094B1A61012901D130BF02E040BFE4
S315080036E020BF20BF044A126904239A43024B1A6179
S315080036F0704700000070004000ED00E010B501F0D2
S3150800370001F940210F48FFF758FC40210920C0065F
S31508003710FFF753FC00210C48FEF716FE00210A4865
S31508003720FEF71EFEFFF770FB01F0ECF80121080713
S3150800373000F01CF801210846FFF7C0FF00F0B4FAB4
S3150800374010BD00000004004800240140002905D0EF
S31508003750054A52690243044B5A6104E0024A526917
S315080037608243014B5A61704700100240002905D078
S31508003770054AD2690243044BDA6104E0024AD26977
S315080037808243014BDA61704700100240002905D0D8
S31508003790054A92690243044B9A6104E0024A926917
S315080037A08243014B9A6170470010024010B500F041
S315080037B031F804494968F02211400909024A515C66
S315080037C0C84010BD00100240FC00002010B5FFF7ED
S315080037D0EDFF05494968072212021140090A034A02
S315080037E0515CC84010BD000000100240FC000020DB
S315080037F010B5FFF7DBFF054949680722D2021140D9
S31508003800C90A034A515CC84010BD000000100240B6
S31508003810FC000020F8B51E4840680C210840042822
S3150800382002D008282ED101E01A4C2DE01848403065
S315080038300069C007C00F00280AD015484030006943
S3150800384002210840002801D0134802E0114800E090
S31508003850104807460E4840300069FF210904084011
S31508003860000C451C0A484030006907210902084037
S31508003870000A461C3946694308463146FEF74AF8A7
S31508003880044601E0034C00BF00BF2046F8BD000017
S315080038900010024000127A0000093D0070B5044687
S315080038A000250221074800F066FC002808D00548D4
S315080038B000F0BAFC20700221024800F054FC0125F1
S315080038C0284670BD0038014010B500F001F810BD5B
S315080038D000B585B062480068012108436049086060
S315080038E000BF5F480068022108400028F9D05D48FB
S315080038F05D4908605D480068102108435B49086017
S3150800390008460068C008C000086057490968481E8C
S315080039105749FDF7FFFF0490544800680499490782
S31508003920490F0843514908604D48406851490840C5
S315080039304B49486008464068902108434849486012
S31508003940084640684860484800684649884207D99A
S3150800395043484068052109020843414948600BE08D
S31508003960414800684449884206D93D4840680121D3
S31508003970890208433A4948606B4601AA3A480168F1
S315080039803E48FEF791FD36484030006980088000C1
S31508003990334940310861084600694008400008611B
S315080039A0684600784007400F02906846007940064E
S315080039B0400E03902A48C069890508432849C8610A
S315080039C02748403000692E4908402549403108619A
S315080039D003980004029909020843214940310969FC
S315080039E008431F49403108611D480068012109063E
S315080039F008431B49086000E000BF19480068012118
S31508003A00490608400028F7D0154840688008800015
S31508003A10134948600846406802210843104948602F
S31508003A2000E000BF0E4840680C2108400828F8D17D
S31508003A300120FEF791FE0A4840681021884308498C
S31508003A4048600120FEF788FE0548406880218843C3
S31508003A50034948600120FEF77FFE05B000BD00005F
S31508003A600010024000A24A040C0100200020024077
S31508003A7000366E010FC0FFFF0051250200127A00C2
S31508003A80FFF800FF042806D10649096904221143F4
S31508003A90044A116105E00349096904229143014A70
S31508003AA01161704700E000E010B5FFF753FC754858
S31508003AB00088401C734908800846C068401CC860D6
S31508003AC071480088401C70490880704800680028C2
S31508003AD004D06E480068401E6C4908606C48007A3D
S31508003AE0012805D167480069401C6649086102E05B
S31508003AF000206449086163483430007A01280ED1F1
S31508003B0060484069401C5F49486108464069614908
S31508003B10884207D900215B483430017202E0002050
S31508003B205849486157483430807A012805D15548A4
S31508003B30C06A401C5349C86202E000205149C86265
S31508003B405348007D002809D04E484068401C4D491E
S31508003B5048600846806A401C886203E0002049499C
S31508003B60486088624A48807904280AD14548C0696D
S31508003B704949884208D24348C069401C4149C8613E
S31508003B8002E000203F49C861FF2101314348FFF7A1
S31508003B900BFA002813D03B483430407800280ED161
S31508003BA03B48007901280AD13648006A39498842D3
S31508003BB008D23448006A401C3249086202E00020F4
S31508003BC0304908622F483430C07A012813D1C1031E
S31508003BD00920C006FFF7F3F92A4881688068401C67
S31508003BE0284A9060FF20F530814225D900211046E9
S31508003BF03430C17220E023483430C07A022812D10A
S31508003C0081030920C006FFF7DAF91E488168806833
S31508003C10401C1C4A9060224881420DD9002110465A
S31508003C203430C17208E00020164988600121C903B2
S31508003C300920C006FFF7C1F91548007D012805D1FE
S31508003C401048006B401C0F49086302E000200D492C
S31508003C5008637E2000F086FE20211048FFF7A4F9AD
S31508003C6000280AD00748406A0E49884208D2054803
S31508003C70406A401C0349486202E000200149486244
S31508003C8010BD0000CC010020280100202C010020D6
S31508003C908C0300208813000050C30000000400486D
S31508003CA0DC050000B888000010B516480068012138
S31508003CB008431449086008464068134908401149F2
S31508003CC0486008460068114908400E4908600846D9
S31508003CD000680121890488430A4908600846406843
S31508003CE0C32109048843074948600846006808490B
S31508003CF00840044908609F2000048860FFF7E4FD37
S31508003D0010BD0000001002400CC0FFF8FFFFF6FED1
S31508003D10FFFF8F0010B50421080700F017F90028E7
S31508003D2006D00421080700F0EBF80121014881704C
S31508003D3010BD00000002002008B501214804FFF765
S31508003D4005FD022201210920C006FFF7E4F8022139
S31508003D50684601801821C1700121817069460920D1
S31508003D60C006FFF78BF808BD10B50121164800F00C
S31508003D70EDF8002827D00121134800F0C1F81348B0
S31508003D80807801281FD11248C179C079401CC2B277
S31508003D900F48C2710B2916DD0C48C078012804D1DA
S31508003DA001020920C006FFF70AF90948C0790D285B
S31508003DB009DD00210548817001210648FEF73AFB16
S31508003DC000210348C17110BD000400400002002014
S31508003DD08C0300200024014030B589B004460D4606
S31508003DE001210846FFF7C2FC06A800F049F9079426
S31508003DF0684605830021018408A881706846817693
S31508003E0006A90120800700F005F90F21684601710F
S31508003E1001214171817101A8FFF7FEFB0421080702
S31508003E2000F06AF801220421080700F09CF802A8AD
S31508003E3000F0DCF860216846017201214172002019
S31508003E40039000216846017402A90120800700F04A
S31508003E5095F80821C80600F0C1F84021080600F0C8
S31508003E606DF80121880700F03BF80121880700F06A
S31508003E7057F80121880700F047F809B030BD00005F
S31508003E807FB504460D4601210220FFF76FFC684600
S31508003E9000F0F6F8019468460580002101818172D8
S31508003EA0817069460D4800F0B5F81021684601731F
S31508003EB0022141730121817303A8FFF7ADFB01219C
S31508003EC0064800F019F801221146044800F04BF89C
S31508003ED00121024800F018F87FBD000000040040E8
S31508003EE0002904D0026880231A43026003E00268AE
S31508003EF080239A430260704702698A4302617047C9
S31508003F0002698A4302617047002904D002680123C6
S31508003F101A43026003E002685208520002607047C2
S31508003F20002905D0426C0123DB031A43426404E0EE
S31508003F30426C0123DB039A43426470478269072374
S31508003F401B039A430B021A438261704702461069A3
S31508003F500840002805D0D0680840002801D0012074
S31508003F6070470020FCE7002A03D0C3680B43C360F0
S31508003F7002E0C3688B43C3607047000010B58269CE
S31508003F8007231B039A430B781B021A4382610A7A9A
S31508003F9012014B781B011A43036A3024A3431A43C0
S31508003FA002624A6882630C4A904213D14A7A120125
S31508003FB08B781B011A43036AC024A3431A4302627F
S31508003FC04A8992008B899B001A4343682401A343BC
S31508003FD01A43426010BD0000002C0140826901238B
S31508003FE0DB029A430B021A43826170470021017073
S31508003FF041708170416001724172418181817047CF
S3150800400001229207904201D1816301E08AB282635C
S3150800401070470000026803231B029A430B891A4360
S315080040200260134A904206D001229207904202D0BB
S31508004030104A904205D1026870239A438B781A4336
S3150800404002600B4A904205D00B4A904202D00B4AB6
S31508004050904205D1026B120A12028B7A1A43026346
S315080040604A68C2620A888262012242617047000079
S31508004070002C014000040040004401400048014073
S315080040800021C9434160002101800181817081724C
S31508004090704710B5FFF758F910BD000070B5FFF767
S315080040A085FB05467D21C900FDF734FC0446601EE4
S315080040B00C49884200D90CE0601E0B49486103216F
S315080040C0081F00F0D5FC0020074988610720086111
S315080040D000BF0420FFF7D6FC0021481E00F0C8FCEC
S315080040E070BD0000FFFFFF0000E000E010B50221F0
S315080040F00A4800F049F800280ED0084800F094F85D
S31508004100C4B20748407A002802D1204602F0FAF8DD
S315080041100221024800F027F810BD000000380140CF
S315080041200002002010B504462146054800F080F834
S3150800413000BF0121024800F01EF80028F9D010BD82
S315080041400038014070B504460D467E2000F00AFC92
S3150800415003E02078641CFFF7E5FF2846691E8DB248
S315080041600028F6D170BD4161704782695208520035
S315080041700A4382617047024690680840002801D0C9
S31508004180012070470020FCE70246D0680840002856
S3150800419001D0012070470020FCE7002A03D00369FC
S315080041A00B43036102E003698B4303617047000018
S315080041B070B504460D460026E06930218843297902
S315080041C00843E061E06944218843A9790843E0612E
S315080041D0E06980088000297A0843E061A06918210F
S315080041E0884369890843A061A06904218843297B1B
S315080041F00843A0610B48844203D1FFF7F9FA064643
S3150800420002E0FFF7E3FA064630462968FDF782FB27
S315080042100009206230462968FDF77CFB0007000F7D
S31508004220606270BD0038014001464868C0B27047F8
S31508004230CAB2026070474B21C90101603021017181
S315080042400021817101721821418100210173704793
S3150800425010B51D484088030000F0FBFB0504111E3D
S315080042602B2C2D0018487C304089FF218A31884242
S3150800427004DC01211448418000F094FB1BE012483D
S315080042807C304089FF216F31884204DC02210E48C8
S31508004290418000F087FB0EE00B487C304089FF2107
S315080042A05531884204DC03210748418000F07AFB37
S315080042B001E000E000BF00BF03487C300079002819
S315080042C001D100F06FFB10BD1003002008B59E4811
S315080042D04088002806D001286ED002287ED0032800
S315080042E069D1DFE0022198487C3081712021974806
S315080042F0FEF75AFE002841D09549C868FF21F531D6
S31508004300FDF708FBC007C00F00281CD110210920A3
S31508004310C006FEF752FE08210920C006FEF74DFE2C
S3150800432000BF202168460180012181701021C170DB
S3150800433069460920C006FEF7A1FD20210920C0060E
S31508004340FEF73BFE37E010210920C006FEF737FED0
S3150800435008210920C006FEF732FE00BF8021684604
S3150800436001800021C17069460920C006FEF786FD56
S3150800437020210920C006FEF722FE1CE01021092094
S31508004380C006FEF71AFE08210920C006FEF715FE2C
S3150800439000BF202168460180012181701021C1706B
S315080043A069460920C006FEF769FD20210920C006D6
S315080043B0FEF703FE00BFC5E0012163487C3081712A
S315080043C020216248FEF7F0FD002817D06049C8682A
S315080043D0FF21F531FDF79EFAC00700E02AE0C00F7D
S315080043E0002805D108210920C006FEF7E6FD0AE0E7
S315080043F008210920C006FEF7E2FD04E0082109208D
S31508004400C006FEF7DAFD10210920C006FEF7D7FD23
S3150800441000BF8021684601800021C17069460920D5
S31508004420C006FEF72BFD20210920C006FEF7C7FDB2
S3150800443000BF87E020214548FEF7B6FD002815D0C5
S315080044404349C868FF21F531FDF764FAC007C00F74
S31508004450002805D110210920C006FEF7B0FD0AE0A4
S3150800446010210920C006FEF7A8FD04E01021092046
S31508004470C006FEF7A2FD08210920C006FEF79FFD2B
S3150800448000BF8021684601800021C1706946092065
S31508004490C006FEF7F3FC20210920C006FEF78FFDB3
S315080044A000BF4FE020212948FEF77EFD002815D0E1
S315080044B02749C868FF21F531FDF72CFAC007C00F58
S315080044C0002805D110210920C006FEF778FD22E054
S315080044D010210920C006FEF770FD1CE01C49C868BB
S315080044E0CD21FDF717FAC007C00F002805D1102106
S315080044F00920C006FEF763FD0DE01549C868CD2101
S31508004500FDF708FAC007C00F002804D010210920BB
S31508004510C006FEF752FD08210920C006FEF74FFD2A
S3150800452000BF8021684601800021C17069460920C4
S31508004530C006FEF7A3FC20210920C006FEF73FFDB2
S3150800454000BF00BF00BF08BD1003002000040048DC
S31508004550CC01002008B50421E54881718079030063
S3150800456000F077FA05045198FEFDFC00E048408902
S31508004570FF218A31884203DB0121DD48817141E050
S31508004580DB484089FF21873188420ADDD8487C38D4
S315080045904088022805D00221D5487C38418000F0A1
S315080045A001FA2021D348FEF7FFFC00282AD0D24979
S315080045B0C868FF21F531FDF7ADF9C007C00F00281F
S315080045C005D110210920C006FEF7F9FC04E01021E8
S315080045D00920C006FEF7F1FC00BF8021684601806D
S315080045E00021C17069460920C006FEF747FC202154
S315080045F00920C006FEF7E3FC00BF08210920C00613
S31508004600FEF7DDFC72E1BA484089FF21A2318842F3
S3150800461003DB0221B64881713BE02021B548FEF74D
S31508004620C3FC002835D0B449C868FF21F531FDF729
S3150800463071F9C007C00F002805D108210920C00656
S31508004640FEF7BDFC04E008210920C006FEF7B5FC0C
S3150800465010210920C006FEF7B2FC00BF802168467B
S3150800466001800021C17069460920C006FEF706FCD4
S3150800467020210920C006FEF7A2FC00BF9C487C3812
S315080046804088012805D0012199487C38418000F0EE
S3150800469089F92BE196484089FF21A531884203DB39
S315080046A003219348817165E020219248FEF77CFC3E
S315080046B000285FD0FF2101318E48FEF775FC0028DF
S315080046C007D08D48006A8D49884202D90421884856
S315080046D081718949C868FF21F531FDF71BF9C007C3
S315080046E0C00F00281CD110210920C006FEF765FC62
S315080046F008210920C006FEF760FC00BF2021684695
S315080047000180012181701021C17069460920C00607
S31508004710FEF7B4FB20210920C006FEF74EFC1AE07E
S3150800472010210920C006FEF74AFC00BF8021684612
S3150800473001800021C17069460920C006FEF79EFB6C
S3150800474020210920C006FEF73AFC00BF08210920EF
S31508004750C006FEF734FC66487C3802E0C5E06DE02A
S3150800476009E04088002805D0002161487C3841804E
S3150800477000F018F9BAE020215E48FEF715FC00287B
S315080047805BD0FF2101315B48FEF70EFC002807D0FD
S315080047905948006A5949884202D904215448817106
S315080047A05549C868FF21F531FDF7B4F8C007C00FB1
S315080047B000281CD110210920C006FEF7FEFB08219F
S315080047C00920C006FEF7F9FB00BF202168460180D4
S315080047D0012181701021C17069460920C006FEF7C3
S315080047E04DFB20210920C006FEF7E7FB1AE0102141
S315080047F00920C006FEF7E3FB00BF8021684601805A
S315080048000021C17069460920C006FEF737FB202142
S315080048100920C006FEF7D3FB00BF08210920C00601
S31508004820FEF7CDFB32487C384088002805D00021A9
S315080048302F487C38418000F0B5F857E020212D48F4
S31508004840FEF7B2FB00284FD029487C38408800285C
S3150800485005D0002126487C38418000F0A3F8264878
S31508004860C069274988421CD210210920C006FEF7D4
S31508004870A4FB08210920C006FEF79FFB00BF2021E4
S3150800488068460180012181701021C170694609209E
S31508004890C006FEF7F3FA20210920C006FEF78DFBB5
S315080048A01AE010210920C006FEF789FB00BF802107
S315080048B0684601800021C17069460920C006FEF7D6
S315080048C0DDFA20210920C006FEF779FB00BF082182
S315080048D00920C006FEF773FB0748343040780128E4
S315080048E002D103210248817100E000BF00BF08BD64
S315080048F08C03002000040048CC010020941100001D
S315080049003075000010B5FEF72BF9FEF787F802F0B0
S315080049104DFB10BD03488068400840000149886087
S3150800492070470000002C004080210143014A1160B5
S3150800493070470000002C004003488068002801D01A
S31508004940012070470020FCE7002C004010B5FFF757
S31508004950F3FF002804D0FFF7DDFF662000F002F819
S3150800496010BD00004106490E014A1160704700005B
S31508004970002C004004494968FF22813291430143D3
S31508004980014A516070470000002C004004494968FC
S31508004990C909C9014206520E1143014A51607047BE
S315080049A0002C004010B57E20FFF7DCFF0948FEF713
S315080049B04FF90949094881800621001D00F03AFD92
S315080049C00649091D8881402202490448001DFEF750
S315080049D07CF910BD00F80008FBAA00000C030020B3
S315080049E070B505460C460121C802FEF7BFFEFF203A
S315080049F08130FFF7BFFF2046FFF7C8FF2846FFF7BD
S31508004A0093FF70BD0FB410B503A9044B044A02986E
S31508004A1000F034F910BC08BC04B01847E16200087D
S31508004A20C80100202021020C01D010211046020ADC
S31508004A3001D010460839020901D01046091F82081C
S31508004A4001D01046891E420801D0881E7047081AF0
S31508004A50704730B47446641E2578641CAB4204D390
S31508004A60635D5B00E31830BC18471D46F8E7000095
S31508004A7010B5002819DB1A4A03231B02D21883082B
S31508004A809B00D2588307DC0EFF23A3409A438B076B
S31508004A901B0E8407E40EA3401A43114B0324240279
S31508004AA01B198408A4001A5118E00E4A03071B0FA5
S31508004AB0083B9B089B00D2588307DC0EFF23A340C4
S31508004AC09A438B071B0E8407E40EA3401A43054B33
S31508004AD00407240F083CA408A4001A5110BD0000BE
S31508004AE000E100E01CED00E002E008C8121F08C162
S31508004AF0002AFAD170477047002001E001C1121F51
S31508004B00002AFBD170470000F0B51FB486B009989B
S31508004B10089A030D0021024314D05148514A181827
S31508004B20504305141198012810981AD0281A401CC9
S31508004B3000264D4F4D49009601910490002812DA3F
S31508004B40444211E01198012449A3012801D1109883
S31508004B50C1430698119A84600360C26041600BB035
S31508004B60F0BD4042E4E70446210500203F4A001C08
S31508004B7051410391029012E0E00707D032463B46C6
S31508004B8001990098FDF778F90191009032463B4665
S31508004B9010461946FDF770F906460F466410002CB4
S31508004BA0EAD10498039B0028029A0999089806DA1C
S31508004BB0FDF762F9019B009AFDF75EF905E0FDF73E
S31508004BC0C3F9019B009AFDF7BFF904460E46002279
S31508004BD0284BFDF705F803D80020C043014607E037
S31508004BE00022254B20463146FDF794F8FDF724FAB6
S31508004BF0102409E0002C0ADB0A220023FDF718F826
S31508004C00079B30321A55641E02460A43F2D1112216
S31508004C10641C079B121B1C19119B012B03D0012333
S31508004C2008430ED10AE0084304D011201090002052
S31508004C30119077E71098151A6D1E0BE010988242AE
S31508004C4002DD00236D1C03E0824201DA00236D1E9B
S31508004C50002BEED0069811998260C16030C07EE7BD
S31508004C6001FCFFFF104D0000000014400000F03F5B
S31508004C70300000000000F0430000E03FFFB597B0A9
S31508004C800646002518E2252877D100242746FD493F
S31508004C90049400E00443761C32780120203A9040C0
S31508004CA00842F7D130782A280ED0022230780146F9
S31508004CB03039092916D804990A2359433039401836
S31508004CC01443761C0490F1E7189802C804911890CA
S31508004CD0002904DA012040030443484204900220D4
S31508004CE00443761C30782E2814D1042004437078A7
S31508004CF0761C2A2809D11898761C80C8189009E0CD
S31508004D000A214F43303FC719761C3078014630399F
S31508004D100929F5D930786C2810D006DC4C281AD029
S31508004D2068280ED06A2817D104E0742813D07A2888
S31508004D3012D110E00120400504430CE001210905C9
S31508004D4001E0032109050C437178814203D1012052
S31508004D5000052418761C761C3078119066280BD02E
S31508004D6013DC58287DD009DC00287BD04528F6D0EE
S31508004D704628F4D047281AD1A5E118E0632835D08B
S31508004D80642870D0652812D19DE170286CD008DCA3
S31508004D906728F1D069287BD06E280DD06F2806D1F8
S31508004DA0BAE073282ED0752871D0782859D01A9A67
S31508004DB0199990476D1C7EE16002400F022809D0C0
S31508004DC003280DD00428189801680DD00D60001D21
S31508004DD0189070E11898EA1701680D604A60F6E7BE
S31508004DE0189801680D80F2E70D70F0E718986A4682
S31508004DF001781172001D18900020507202A80090C8
S31508004E00012005E0189802C8189000200091C043B8
S31508004E1061070DD5002101E00199491C0191B942AC
S31508004E2012DA8142F8DB009A515C0029F4D10BE0D2
S31508004E30002101E00199491C01918142FADB019A9E
S31508004E400099895C0029F5D1019904981A9B471A9B
S31508004E5021463846199A00F097FA019940194518DB
S31508004E600BE04FE02CE113E04EE000980099007843
S31508004E70491C00911A9A199990470198401E019069
S31508004E80401CF2D1214638461A9B199A10E137E0A0
S31508004E900A200021009001916002410F022907D0E3
S31508004EA0189A01CA1892C2179446032908D00AE02C
S31508004EB01898C01DC108C90005C91891944607E08D
S31508004EC000B2C2179446042902D140B2C1178C46D3
S31508004ED000226146944506DA0A460021404291417D
S31508004EE08C462D2102E0210504D52B216A46117333
S31508004EF0012103E0E10701D02021F7E7029155E0FF
S31508004F000A200AE0102008E0102000900021042062
S31508004F1004430191082703E008200021019100902D
S31508004F206002410F022907D0189A01CA1892002276
S31508004F309446032908D008E01898C01DC108C9007E
S31508004F4005C91891944603E080B2042900D1C0B27D
S31508004F5000210291210729D51199702906D0009AB6
S31508004F601021019B4A401A4305D00EE040216A46AB
S31508004F701173012108E06146014306D030216A46D3
S31508004F8011731199517302210291009A0821019B0C
S31508004F904A401A430AD16146014301D1610705D542
S31508004FA030216A46117301217F1E029111995829F1
S31508004FB004D035A10E910DA90D910DE037A1F9E7A1
S31508004FC06146019B009AFCF733FE0E9B8C469B5C60
S31508004FD00D9A521E0D92137061460143F0D10D9839
S31508004FE005A9081A20300190600703D5012000049E
S31508004FF0844300E001270198874201DD381A00E062
S315080050000020019900904118029809180498401A3E
S315080050100490E00306D421461A9B199A049800F0D6
S31508005020B3F94519002706E003A81A9AC05D19992D
S3150800503090476D1C7F1C02988742F5DBE0030CD570
S3150800504021461A9B199A049800F09EF9451904E01E
S315080050501A9A3020199990476D1C0099481E00909D
S315080050600029F5DC08E00D980D990078491C0D918A
S315080050701A9A199990476D1C0199481E01900029A2
S31508005080F1DC63E109280100303132333435363733
S315080050903839616263646566000000003031323376
S315080050A03435363738394142434445460000000016
S315080050B000F05AF94519761C3078002800D0E2E548
S315080050C028461BB0F0BD600700D406271898C01DF7
S315080050D0C108C90048680A680831C30FDB07189178
S315080050E0190001D09CA108E0210501D59BA104E087
S315080050F0E10701D09AA100E09AA1430011985B0844
S31508005100109165280CD006DC452809D046281DD004
S31508005110472841D141E0662818D067283CD13CE0B1
S315080051200021112F01DB112000E0781C019100906D
S3150800513008A911A8FFF7E8FC139905910021119A0F
S3150800514015927F1C12980197009150E00120C00724
S3150800515003900120019008A9009711A8FFF7D4FC35
S31508005160139A149905920022119B0092129815938E
S31508005170059A0192002901D0104602E0791C4018D0
S315080051800190381A01D5019804E04042401E00906B
S31508005190781C0190C01B029043E0012F00DA01271A
S315080051A00021112F01DD112000E038460191009001
S315080051B008A911A8FFF7A8FC13990591119A0021CF
S315080051C0129815920091019721070CD40599B942B6
S315080051D001DB019900E00191012904DD159A491EB8
S315080051E0515C302906D0B84201DA011D05DA0121E1
S315080051F0029115E00199491EEDE7002805DC0099A2
S31508005200411800910199091A03E0019A411C91423B
S3150800521000DD01910099401A401C02900120C00748
S315080052200390200706D402990198814202DB0020E8
S31508005230C043029000206946C87707AF012103984A
S315080052400337C907884224D0022011902B201290D8
S31508005250039800280CDA404203902D20129007E0AC
S315080052600A210398FCF756FB30317F1E03903970EC
S315080052701199481E11900029F2DC03980028EFD1F5
S31508005280791E129808703078202108404530BF1ED4
S31508005290387006A8C01BC01D039010980078002817
S315080052A000D00120019941180298C01709180398DF
S315080052B009180498401A401E0490E00306D42146B3
S315080052C01A9B199A049800F05FF845191098007807
S315080052D0002803D01A9A199990476D1CE00324D523
S315080052E021461A9B199A049800F04EF845191CE0B5
S315080052F00098002807DB00990598884203DD159871
S31508005300405C199901E0199930201A9A904700983B
S315080053106D1C401C00900298401E0290002804D183
S315080053201A9A2E20199990476D1C0199481E0190CA
S315080053300029DDDC05E038781A9A7F1C1999904710
S315080053406D1C0399481E03900029F4DC21461A9B1C
S31508005350199A0498ACE600002D0000002B00000006
S315080053602000000000000000F8B5044600251E468F
S315080053701746880404D405E039462020B0476D1C3A
S31508005380641EF9D52846F8BDFFB50446002581B048
S315080053901E46C80301D5302700E02027880404D517
S315080053A005E038460399B0476D1C641EF9D52846B2
S315080053B005B0F0BD10B51948007801282DD1002098
S315080053C0164908701649088012E0154800884000FA
S315080053D01449085A14490988C900144A8918104AF0
S315080053E01288520088520E480088401C0C490880D2
S315080053F00B4800880428E8DB7E20FFF7B3FA0A4842
S315080054000088401C0849088008460088142804DBE0
S315080054100020088001200649087010BD5C010020A4
S315080054207201002028040020740100206004002076
S315080054305401002010B502460023002901D100209E
S3150800544010BD03E01488921CE01883B208464C1E6F
S31508005450A1B20028F6D11846F2E7000010B5FEF70B
S3150800546023FCFDF783FFFEF793F8FDF7AFF9FCF78A
S315080054703BFF0B20FCF7A6FE0C20FCF7A3FE03203F
S31508005480FCF7A0FE0420FCF79DFE01212048FCF74E
S31508005490D1FFE1204002FDF7DDF801211D48017129
S315080054A0002101754171FF388D38417181710121E3
S315080054B018484172FDF78CFFFEF73EFC164963203B
S315080054C0FEF78AFC1A216320FEF7DAFCFEF7E6FDF2
S315080054D010487C384089002801D1FEF7F7FE7F2165
S315080054E07E20FFF77DFA00210C48417040210920F3
S315080054F0C006FDF764FD40210948FDF760FDFFF78A
S3150800550001FA00200749087004493439C86010BDFB
S31508005510002401408C030020581B000000020020D4
S3150800552000040048C400002070B50025A748807A0A
S3150800553001280ED1A5483438C06AFF21F5318842C2
S3150800554007D90021A14881720020A1490880A149F4
S3150800555008709E48407A012870D19D48007A012833
S3150800556011D003280ED19C48007D002806D1974803
S31508005570007A002802D1012194480172002093493B
S31508005580343948611BE19248407A07286FD007DC16
S315080055900300FFF75EFA0712235685839596830064
S315080055A00A2879D004DC082877D0092876D1B0E013
S315080055B0A12874D0A528F9D1FBE000208349343905
S315080055C0486101218148C171002202218348FEF702
S315080055D0E4FD00207D493439C860EEE000207B49AF
S315080055E0343948617A48807A012811D17848007B95
S315080055F0282825DA7648007B0A2821DD7448017BAD
S31508005600724810304181012110388173C17017E04A
S315080056106F48807A022812D16D4A117BD07A00F041
S315080056202FFF0546282D0BDA0A2D09DD67481030AD
S315080056304581012110388173C17001E0C3E070BD56
S31508005640BBE000206149343948616148807A022804
S3150800565021D15F4A117BD07A00F012FF012807D1C9
S3150800566003215D4801755EA0FFF7CCF913E038E029
S31508005670574A117BD07A00F003FF00280BD100218E
S31508005680554801755148C07B012804D100F0ECFD4E
S3150800569000214E48C17390E082E032E08CE085E05C
S315080056A04B48807A02280AD1494A117BD07A00F001
S315080056B0E7FE46491031C88001214448C1737CE0A1
S315080056C07BE00020414934394861414A117BD07A50
S315080056D000F0D6FE3D4910314880012001F0BCFAA1
S315080056E06BE00020394934394861394A117BD07A50
S315080056F000F0C6FE354910318880032001F0ACFA67
S315080057005BE00020314934394861022001F0A4FAEF
S3150800571053E000202D49343948612D49887AC1174C
S31508005720890F091889108900411A33D12849887ABE
S31508005730C117890F09188910244A10321181104699
S3150800574000891C2826DA00241FE0A200921D204B9F
S315080057509B1D995CA200521D985C00F091FE0146C3
S31508005760A2001A481E308152A2000832184B9B1D0F
S31508005770995CA200D21D985C00F082FE0146A20048
S3150800578012481E3010184180641C104810300089D9
S31508005790A042DADC042001F05FFA00F065FD0CE0B7
S315080057A0052001F059FA00F05FFD06E001F01CFA49
S315080057B003E001F0B5F900E000BF00BF00BF00BF7D
S315080057C000210248417200BF39E7000000020020AC
S315080057D000050020C40100208C0300200038014089
S315080057E00A484F545F310A0070B505460C46002D2D
S315080057F002D0012D1ED10CE0602101208007FEF7A2
S315080058009DFB002101208007FEF7FAFB0A48047079
S3150800581010E009480078A04209D0602101208007DD
S31508005820FEF78CFB214601208007FEF7E9FB0248BC
S31508005830047000BF00BF70BD7701002008B5FE48A0
S315080058400079012879D1FD48007D0028FAD1FA4867
S3150800585040790300FFF7FDF808050772D8F1F0EF65
S31508005860EEED002008BDF5492039C868FF219131C1
S31508005870FCF750F88007800F00280AD1102109206C
S31508005880C006FDF79CFB08210920C006FDF797FB1B
S3150800589040E0EA492039C868FF219131FCF73AF817
S315080058A08007800F01280AD110210920C006FDF7BC
S315080058B084FB08210920C006FDF781FB2AE0DF49A1
S315080058C02039C868FF219131FCF724F88007800F3A
S315080058D002280AD110210920C006FDF770FB08210D
S315080058E00920C006FDF76BFB14E0D4492039C868C7
S315080058F0FF219131FCF70EF88007800F032809D1A4
S3150800590008210920C006FDF758FB10210920C0060A
S31508005910FDF755FB00BF8021684601800021C17054
S3150800592069460920C006FDF7A9FA20210920C00604
S31508005930FDF745FB00BF012094E7E2E1BF492039A6
S31508005940C868C821FBF7E6FF8007800F00280AD140
S3150800595010210920C006FDF732FB08210920C006E0
S31508005960FDF72DFB3DE0B5492039C868C821FBF78E
S31508005970D1FF8007800F01280AD110210920C0060F
S31508005980FDF71BFB08210920C006FDF718FB28E0D8
S31508005990AA492039C868C821FBF7BCFF8007800FD1
S315080059A002280AD110210920C006FDF708FB0821A4
S315080059B00920C006FDF703FB13E0A0492039C86893
S315080059C0C821FBF7A7FF8007800F032809D1082104
S315080059D00920C006FDF7F1FA10210920C006FDF7D7
S315080059E0EEFA00BF8021684601800021C170694631
S315080059F00920C006FDF742FA20210920C006FDF756
S31508005A00DEFA00BF01202DE78C492039C868C82175
S31508005A10FBF780FF8007800F00280FD1102109208F
S31508005A20C006FDF7CCFA08210920C006FDF7C7FA1B
S31508005A3042E065E12FE1C4E08AE050E07F49203981
S31508005A40C868C821FBF766FF8007800F01280AD1BE
S31508005A5010210920C006FDF7B0FA08210920C00662
S31508005A60FDF7ADFA28E075492039C868C821FBF763
S31508005A7051FF8007800F02280AD110210920C0068D
S31508005A80FDF79DFA08210920C006FDF798FA13E0EC
S31508005A906A492039C868C821FBF73CFF8007800F90
S31508005AA0032809D108210920C006FDF786FA102126
S31508005AB00920C006FDF783FA00BF802168460180E9
S31508005AC00021C17069460920C006FDF7D7F92021D3
S31508005AD00920C006FDF773FA00BF0120C2E6574940
S31508005AE02039C868FF212D31FBF714FFC007C00F06
S31508005AF0002805D110210920C006FDF760FA0FE03D
S31508005B004E492039C868FF212D31FBF703FFC0072E
S31508005B10C00F002804D010210920C006FDF74DFA51
S31508005B2000BF8021684601800021C17069460920AE
S31508005B30C006FDF7A3F920210920C006FDF73FFAA4
S31508005B4000BF08210920C006FDF739FA012089E6B9
S31508005B503A492039C868FF219131FBF7DBFEC007B7
S31508005B60C00F002805D110210920C006FDF727FA25
S31508005B700FE032492039C868FF219131FBF7CAFE88
S31508005B80C007C00F002804D010210920C006FDF761
S31508005B9014FA00BF8021684601800021C170694659
S31508005BA00920C006FDF76AF920210920C006FDF77D
S31508005BB006FA00BF08210920C006FDF700FA0120F1
S31508005BC050E61E492039C868C821FBF7A3FE80079E
S31508005BD0800F00280AD110210920C006FDF7EFF929
S31508005BE008210920C006FDF7EAF941E013492039E2
S31508005BF0C868C821FBF78EFE8007800F01280AD1E6
S31508005C0010210920C006FDF7D8F908210920C00689
S31508005C10FDF7D5F92CE009492039C868C821FBF7F2
S31508005C2079FE8007800F02280FD110210920C006AF
S31508005C30FDF7C5F9082103E08C030020EC010020DC
S31508005C400920C006FDF7BBF912E02F49C868C8212C
S31508005C50FBF760FE8007800F032809D10821092079
S31508005C60C006FDF7AAF910210920C006FDF7A7F915
S31508005C7000BF8021684601800021C170694609205D
S31508005C80C006FDF7FBF820210920C006FDF797F9A5
S31508005C9000BF0120E6E51C49C868C821FBF73AFEA3
S31508005CA0C007C00F002805D110210920C006FDF73E
S31508005CB086F90DE01449C868C821FBF72BFEC00712
S31508005CC0C00F002804D010210920C006FDF775F979
S31508005CD000BF8021684601800021C17069460920FD
S31508005CE0C006FDF7CBF820210920C006FDF767F9A5
S31508005CF000BF08210920C006FDF761F90120B1E5BA
S31508005D0000BF00BFAEE50000CC01002008B5FC4886
S31508005D10007D002838D0FB48C078012834D1F948DE
S31508005D203438C068F84988420ED9F548808964280D
S31508005D300ADAF3484079002806D10721F04841716C
S31508005D400020F0493439C860ED48007D03281BD08F
S31508005D50EB488089FF21EB31884215DDE8488189C7
S31508005D60EAA0FEF74FFEE648407900280CD1E54840
S31508005D703438C068EA49884206D90321E0484171A7
S31508005D800020E0493439C860DD48007901287DD112
S31508005D90DB4840790300FEF75CFE0805074E97DDF1
S31508005DA0FEFDFCFB002008BDD6483438C068E1215A
S31508005DB0C900884239D908210920C006FDF7FFF82D
S31508005DC000BF8021684601800021C170694609200C
S31508005DD0C006FDF753F820210920C006FDF7EFF8A5
S31508005DE000BF10210920C006FDF7E9F80121C548C2
S31508005DF01438017514308079002807D1C14934391F
S31508005E00C8600021BE48017141710AE0BD483438B6
S31508005E10C068AF210901884203D90020B94934393D
S31508005E20C8600121B748417103E00021B54814381C
S31508005E3001750120B7E7B3483438C068B9498842C4
S31508005E403CD908210920C006FDF7B9F800BF802112
S31508005E50684601800021C17069460920C006FDF721
S31508005E600DF820210920C006FDF7A9F800BF10216A
S31508005E700920C006FDF7A3F80121A24814380175C8
S31508005E801430807900280DD19E4900E09CE1343910
S31508005E90C86000219A480171417100209949343936
S31508005EA0C8600FE097483438C068AF2109018842B6
S31508005EB008D9002093493439C86003E00021914885
S31508005EC01438017501206EE78E483438C068964943
S31508005ED0884239D908210920C006FDF770F800BFA5
S31508005EE08021684601800021C17069460920C006E4
S31508005EF0FCF7C4FF20210920C006FDF760F800BFA3
S31508005F0010210920C006FDF75AF801217D481438EA
S31508005F1001751430807900280BD17A493439C86064
S31508005F200021774801714171002076493439C860EB
S31508005F300EE074483438C0687C49884208D9002085
S31508005F4070493439C86003E000216E481438017579
S31508005F50012028E76B483438C0687D21090188424A
S31508005F603ED908210920C006FDF729F800BF80217F
S31508005F70684601800021C17069460920C006FCF701
S31508005F807DFF20210920C006FDF719F800BF03E0B0
S31508005F9019E1D4E072E029E010210920C006FDF7D6
S31508005FA00EF80121574814380175143080790028F5
S31508005FB00BD154493439C8600021514801714171E7
S31508005FC0002050493439C8600EE04E483438C0685D
S31508005FD05349884208D900204A493439C86003E041
S31508005FE000214848143801750120DCE64548343854
S31508005FF0C068E121C90088423AD908210920C006AB
S31508006000FCF7DDFF00BF8021684601800021C170D2
S3150800601069460920C006FCF731FF20210920C00681
S31508006020FCF7CDFF00BF10210920C006FCF7C7FF0B
S3150800603001213448143801751430807900280BD1B1
S3150800604030493439C86000212D480171417100205A
S315080060502C493439C8600FE02A483438C068AF2163
S315080060600901884208D9002026493439C86003E066
S315080060700021244814380175012094E62148343853
S31508006080C0682A49C839884254D908210920C00657
S31508006090FCF795FF00BF8021684601800021C1708A
S315080060A069460920C006FCF7E9FE20210920C0063A
S315080060B0FCF785FF00BF10210920C006FCF77FFF0B
S315080060C001211048143801751430807900280BD145
S315080060D00C493439C8600021094801714171002012
S315080060E008493439C86028E006483438C068104979
S315080060F0884222D9002003493439C8601DE00000CF
S315080061008C03002000020020204E00000A675F77FB
S315080061106F726B2E74656D705F313A25640A0000E4
S31508006120B80B0000A4060000C4090000AC0D00006E
S31508006130CC100000002125480175012033E62348CC
S315080061402038C0682249884238D908210920C00663
S31508006150FCF735FF00BF8021684601800021C17029
S3150800616069460920C006FCF789FE20210920C006D9
S31508006170FCF725FF00BF10210920C006FCF71FFF0A
S315080061800121124801751430807900280BD10F4976
S315080061902039C86000210F480171417100200B4960
S315080061A02039C8600DE009482038C0680A49884285
S315080061B007D9002005492039C86002E000210348B4
S315080061C001750120EFE500BF00BFECE5EC010020FA
S315080061D0A40600008C0300208C0A000010B50524D4
S315080061E016E0FF2101311F48FBF7D7FBFF210131DC
S315080061F01C48FCF793FBFE211A48FCF781FA014676
S315080062001848C030C08F814202D100F06BFC10BD27
S315080062102046611ECCB20028E3D1052416E0FF21F2
S3150800622001311048FBF7B9FBFF2101310D48FCF796
S3150800623093FBFE210B48FCF763FA01460948C03078
S31508006240C08F814202D100F04DFCE0E72046611E76
S31508006250CCB20028E3D100F0CFF900F005F800BF72
S31508006260D5E700001002002010B5FCF7DBFC1A4940
S315080062701A488180001D00891C2815DA1748001D58
S3150800628001890E30FCF7B6F91449091D088908E09A
S315080062900022830011491231CA52830059184A80D4
S315080062A0401C1E28F4D300E010BDFE210B48001D3B
S315080062B0FCF726FA01460948C430C187FF21013197
S315080062C0C038FCF785FBFF2101310448001DFCF7A7
S315080062D08BFB00BFE8E70000FBAA00000C020020C9
S315080062E070B504460D46E1B20548FDF7A1FF00BFAB
S315080062F001210348FDF73FFF0028F9D0204670BD6D
S315080063000038014070B504460025012159488172BC
S31508006310002058493439C86257480088FA2804DDED
S3150800632000205549088055490870544800780300EC
S31508006330FEF78FFB08051D2B3F4B586D799CAA2C41
S315080063400DD101204D4908704B4801880088401C32
S31508006350494A1080901D445400201146C870BB2C31
S3150800636004D101210920C006FCF727FE7FE0FB2C9B
S315080063700AD1414801880088401C3F4A1080901D78
S31508006380445402203D49087071E0012C03D10320D2
S315080063903A49087004E0032C02D1062037490870F0
S315080063A0354801880088401C334A1080901D4454A3
S315080063B05DE0314801880088401C2F4A1080901DF6
S315080063C0445404202D49087051E02B4884700188F4
S315080063D00088401C284A1080901D445405202749EF
S315080063E0087044E02448C078401CC0B22249C870EE
S315080063F08978884202DB0620204908701E480188F1
S315080064000088401C1C4A1080901D44542FE01A48EE
S3150800641001880088401C184A1080901D44540720A3
S315080064201649087023E0144801880088401C124A5F
S315080064301080901D4454801F0188801DFCF760F968
S31508006440002809D100210B488172012141720020E0
S315080064500A4908700849088007480088FA2804DDB0
S315080064600020054908800549087000E000BF00BF04
S3150800647070BD00000002002000050020C4010020B5
S3150800648070B50246002013460C461D02FF2636024A
S3150800649035402543284670BD86B004460D46266815
S315080064A06768A0680590E0680490206903906069B1
S315080064B00290A0690190E069009017A0FEF7A2FA81
S315080064C031461BA0FEF79EFA39461CA0FEF79AFA3B
S315080064D01DA00599FEF796FA1EA00499FEF792FAF2
S315080064E01FA00399FEF78EFA20A00299FEF78AFAF2
S315080064F023A00199FEF786FA26A00099FEF782FAEC
S315080065002948416A29A0FEF77DFA29462BA0FEF7FD
S3150800651079FA00BFFEE700005B4861726420666195
S31508006520756C742068616E646C65725D0D0A000096
S315080065305230203D2025780D0A0000005231203DBA
S315080065402025780D0A0000005232203D2025780DBE
S315080065500A0000005233203D2025780D0A0000006D
S31508006560523132203D2025780D0A000053746163AC
S315080065706B6564204C52203D2025780D0A000000EA
S31508006580537461636B6564205043203D2025780D64
S315080065900A000000537461636B65642050535220EF
S315080065A03D2025780D0A000000ED00E05343425FC8
S315080065B053484353523D25780D0A000043757272BD
S315080065C0656E74204C52203D2025780D0A00000087
S315080065D00749084881800021001D41805F21C900C4
S315080065E0C180152181805F21018100214181704789
S315080065F0FBAA00000C03002000201D4A1D498A80C2
S31508006600F022091D4A8014228A8002220A81192250
S315080066104A81194A8A819200CA8000BF0FE0002287
S31508006620830014498A31CA52830059184A80830064
S3150800663010491231CA52830059184A80401C1C2836
S31508006640EDDB00220B49091DCA81FF225F320A824F
S3150800665014224A82FF225F328A8200228031CA804F
S31508006660891D4A8014228A80FF225F32CA807047B9
S31508006670FBAA00000C020020EE02000008B57E20EE
S31508006680FEF770F9FFF7DAF8012800D108BD8C4843
S31508006690007901287ED18A48007D002802D0012889
S315080066A079D13FE020218748FCF77EFC00282ED1CF
S315080066B08548C0698549884233D28348C0687D21A8
S315080066C0090188422DD27E487C384089002802D1AB
S315080066D0FDF7FCFD25E010210920C006FCF76FFC3C
S315080066E000BF8021684601800021C17069460920E3
S315080066F0C006FCF7C3FB20210920C006FCF75FFC97
S3150800670000BF08210920C006FCF759FC09E06E48BD
S31508006710406A6E49884202D2FDF7D8FD01E0FDF7CE
S3150800672019FFCAE06849C868FF21F531FBF7F2F896
S31508006730C007C00F00281CD110210920C006FCF78D
S315080067403CFC08210920C006FCF737FC00BF2021C5
S3150800675068460180012181701021C17069460920AF
S31508006760C006FCF78BFB20210920C006FCF725FC98
S315080067701DE010210920C006FCF721FC00BF80217E
S31508006780684601800021C17069460920C006FCF7E9
S3150800679075FB01E092E00BE020210920C006FCF71A
S315080067A00EFC00BF08210920C006FCF708FC84E09F
S315080067B04348007D052842D14349C868FF21F53181
S315080067C0FBF7A8F8C007C00F00281CD11021092024
S315080067D0C006FCF7F2FB08210920C006FCF7EDFB12
S315080067E000BF202168460180012181701021C170F7
S315080067F069460920C006FCF741FB20210920C0068E
S31508006800FCF7DBFB58E010210920C006FCF7D7FB94
S3150800681000BF8021684601800021C17069460920B1
S31508006820C006FCF72BFB20210920C006FCF7C7FB96
S3150800683000BF08210920C006FCF7C1FB3CE0204840
S31508006840007D06281BD110210920C006FCF7B7FBDE
S3150800685000BF8021684601800021C1706946092071
S31508006860C006FCF70BFB20210920C006FCF7A7FB96
S3150800687000BF08210920C006FCF7A1FB1CE0102177
S315080068800920C006FCF799FB08210920C006FCF779
S3150800689094FB00BF202168460180012181701021E8
S315080068A0C17069460920C006FCF7E8FA20210920CC
S315080068B0C006FCF782FB00BF00BF00BF00BFE5E6CD
S315080068C08C03002000040048CC010020307500002D
S315080068D008B5FDF7E9F9FCF749FDFCF759FEFBF7A2
S315080068E075FFFBF701FD0C20FBF76CFC0920FBF795
S315080068F069FC0820FBF766FC0720FBF763FC01210F
S315080069005D48FBF797FDE1204002FBF7A3FE012156
S315080069105A48017100214171FF388D3841718171E2
S31508006920012156484172FCF753FDFDF705FA544913
S315080069306320FDF751FA1A216320FDF7A1FAFFF744
S315080069404DFCFDF7ABFB00F0A7F84C487C384089B6
S31508006950002801D1FDF7BAFC00214A4841704021C0
S315080069600920C006FCF72BFB40214748FCF727FB0C
S31508006970FDF7C8FF00214348C171FCF781FE0121DC
S315080069800920C006FCF719FB74E03E483438C06895
S315080069903E49884204D901210920C006FCF70FFBAD
S315080069A03848C079002802D001285ED10AE0FEF7EF
S315080069B0BBFDFBF767FDFFF761FEFCF709FD00F07D
S315080069C01BFB56E00021084600F072F92D483438C2
S315080069D0C0682F49884208D900212A48C171012276
S315080069E002212C48FDF7D9FB39E026493439C86815
S315080069F0FF21F531FAF78EFFC007C00F00281BD11B
S31508006A0010210920C006FCF7DAFA00BF8021684683
S31508006A1001800021C17069460920C006FCF72EFADC
S31508006A2020210920C006FCF7CAFA00BF0821092060
S31508006A30C006FCF7C4FA12E000BF202168460180B0
S31508006A40012181701021C17069460920C006FCF732
S31508006A5015FA20210920C006FCF7AFFA00BFFBF79C
S31508006A6075FD7E20FDF77EFF03E000210548C17114
S31508006A7000BF00BF89E70000002401408C03002006
S31508006A80581B00000002002000040048DC05000036
S31508006A90204E00000038014010B540210F48FAF793
S31508006AA07CFF40210D48FBF775FF06210B48FEF7D2
S31508006AB0C1FC0A49898988420AD10848001F80888A
S31508006AC00749884208D0FFF783FDFDF76BFF03E00F
S31508006AD0FFF77EFDFDF766FF10BD000010030020DE
S31508006AE0FBAA000010B500240C484089052803DBE2
S31508006AF00A484089282803DD1921084841810124CC
S31508006B00064800891D2803DD012402210348018166
S31508006B10012C01D1FFF7A8FB10BD000010020020D0
S31508006B2070B5A0B00025002680216846FAF735FF23
S31508006B30AA2168460170FB21417001218170A521B7
S31508006B40C1701248007A8006010E68460171027902
S31508006B500E490E31401DFAF707FF68460079411DB8
S31508006B606846FBF7CDFD0446211268460079401DAC
S31508006B706A46115468460079801D1454684600799F
S31508006B80C11D6846FDF7DEFA20B070BD1002002070
S31508006B9030B5A1B00446802101A8FAF7FEFE00250B
S31508006BA0AA2168460171FB214171022181710121E7
S31508006BB0C17102210172FF200002204001126846BD
S31508006BC041728472072101A8FBF79AFD0546FF204A
S31508006BD00002284001126846C1720573092101A8FE
S31508006BE0FDF7B0FA21B030BDF0B5A1B000260027F8
S31508006BF0802101A8FAF7D1FE0025AA21684601716D
S31508006C00FB21417101218171A121C1710621017206
S31508006C100FA5027A29460930FAF7A6FE6846007AD1
S31508006C20411D01A8FBF76CFD044621126846007A4F
S31508006C30401D01AA11546846007A801D14546846FE
S31508006C40007AC11D01A8FDF77DFA21B0F0BD00004C
S31508006C504E5F56325F31000030B5A1B00446802140
S31508006C6001A8FAF79AFE0025AA2168460171FB21B8
S31508006C704171022181710521C17102210172FF2032
S31508006C80000220400112684641728472072101A859
S31508006C90FBF736FD0546FF2000022840011268462C
S31508006CA0C1720573092101A8FDF74CFA21B030BD60
S31508006CB070B504460D460026002D13D10846FEF78A
S31508006CC093FD0021AD480182FF388D3841730020BD
S31508006CD0AB498862AB490870A94908630021A748EF
S31508006CE0418249E1A6483430407B00287BD1A4483C
S31508006CF0806AFF21F53188426ED90020A049886252
S31508006D009E48018A8089814210DD9C48018A9EA09E
S31508006D10FDF778FE01219A483430417397488189F6
S31508006D2001827D20C0009E4908800EE09348818933
S31508006D3020461430814208DD924800780F2804DD89
S31508006D4090480078401F8F4908708C4881892046F2
S31508006D502838814234DA89487C384088002803D1AB
S31508006D6048208849087010E084487C384088012803
S31508006D7003D151208349087007E080487C38408851
S31508006D80022802D15A207F4908707D48006B854940
S31508006D9088421ED900207A4908637848418A808942
S31508006DA0814209DB75484079002805D107217348D7
S31508006DB0417100207249C86070488189418208E0A3
S31508006DC0704800780F2804DD6E480078001F6D496A
S31508006DD008706A48818901826A4801780120FEF7AD
S31508006DE003FDC9E0FFE76648806A6D49098888425D
S31508006DF062D90020624988626048018A8089814296
S31508006E005BDA5E48818920461438814215DAFF200C
S31508006E10F5306349088059488189008A081A042888
S31508006E2005DA58480078801C5649087035E05548F8
S31508006E300078401C534908702FE050488189204645
S31508006E400A38814215DAFF20F530554908804B4843
S31508006E508189008A081A022805DA4A480078401CFF
S31508006E604849087019E047480078801E4549087067
S31508006E7013E042488189601F81420EDAFF20F5300F
S31508006E80474908803D488189008A081A022804DB98
S31508006E903C480078801E3B49087038488189018241
S31508006EA08089A04254DD7D20C0003D4908803548D0
S31508006EB00078401E334908704AE030488089A0426D
S31508006EC018DD2E488089001B052809DD7D20C000B5
S31508006ED0334908802B480078801E2A49087034E018
S31508006EE07D20C0002E49088026480078401E254986
S31508006EF008702AE021488089A04226D01F48818947
S31508006F00008A081A052805DD1E480078801C1D49D8
S31508006F1008701AE019488189601F814209DAAF2092
S31508006F2080001F49088017480078801C154908709A
S31508006F300BE01D481A49088010488089A04204DAE7
S31508006F4010480078401C0F4908700C488189018256
S31508006F500C4800780A2803DA0A200A49087006E06D
S31508006F60084800783C2802DD3C2006490870054898
S31508006F7001780120FEF738FC70BD00008C03002064
S31508006F80CC010020F60000200A675F776F726B2E2F
S31508006F906C6173745F74656D703A25640A0000004D
S31508006FA0F8000020B80B0000DC05000008B5012138
S31508006FB04804FCF7CBFB01218804FCF7C7FB6846AD
S31508006FC0FBF7FFFF0421684601804821C170694626
S31508006FD00920C006FBF752FF6846FBF7F2FF20219F
S31508006FE0684601800421C17069460248FBF746FFDE
S31508006FF008BD00000004004838B50024FEF786FEE8
S3150800700001280CD1E648C068FF21F531884205D928
S315080070100121C9030920C006FBF7CFFF38BDE148A7
S31508007020007900287BD101210920C006FBF7C5FF9E
S315080070300020DD49087000210846FFF739FE0021C7
S31508007040D7483430C1701438017508210920C006A4
S31508007050FBF7B5FF00BF8021684601800021C1709B
S3150800706069460920C006FBF709FF20210920C0064A
S31508007070FBF7A5FF00BF10210920C006FBF79FFFFD
S315080070800021C8480175C648C068FF21F531884205
S3150800709009D2C34834304079002803D10121C048B9
S315080070A03430C1726EE10021BD4834304171343844
S315080070B0C068BE498842F5D9BA48407A00280FD137
S315080070C0B748C0687D214901884201D2FDF7C0F85A
S315080070D00021B44841717D204001B149C8600CE0E7
S315080070E0B048007A012808D10020AD49C8600021BF
S315080070F0AC4841710175012101712021AC48FBF7AB
S3150800710053FF002806D00021A64801750121017108
S3150800711038E104E0FCF7F2FAFEF7A0F932E1A148FB
S31508007120007D0300FDF795FC07057797B8C1CAFEF1
S31508007130760000210846FFF7BBFD99483430807B6E
S31508007140002804D1002196483430C17003E001219B
S3150800715093483430C17092483430C07B012808D136
S3150800716094A0FDF74FFCFFF77FF800218C483430D8
S31508007170C1738B48C068914988423CD900208A4926
S31508007180087087483430007A002843D1202188487F
S31508007190FBF70AFF00282AD108210920C006FBF7B9
S315080071A00EFF00BF8021684601800021C170694634
S315080071B00920C006FBF762FE20210920C006FBF75E
S315080071C0FEFE00BF10210920C006FBF7F8FEFDF7FA
S315080071D03FF87E20FDF7C6FB1E20FBF7ADFAFCF74D
S315080071E08DFA00206E49C860FEF738F912E00020D3
S315080071F06B49C8600EE06A48C068FF21F5318842CD
S3150800720008D968487C384089002803D10021644899
S315080072103430C172B5E0012161483430C17060492B
S31508007220C8687D21C900FAF775FB5D49443189882C
S31508007230884206D902215B4801750121FF388D383D
S31508007240C1725749C86800F0BDF8044601212046B6
S31508007250FFF72EFD95E0012151483430C1705049A1
S31508007260C86800F0AFF8044601212046FFF720FD64
S315080072704B49C8687D21C900FAF74CFB4849443197
S3150800728049880F39884206D9012145483430C172E8
S3150800729005214448017574E0012141483430C17024
S315080072A0FF204130FFF704FD6BE001213C483430F4
S315080072B0C17000210846FFF7FBFC62E0012138484F
S315080072C03430C1703438C16844304088401E7D224D
S315080072D0D2005043FF30F530814209D23049C868A0
S315080072E000F070F8044601212046FFF7E1FC2BE088
S315080072F000210846FFF7DCFC012129483430C17219
S315080073003438C16844304088401E7D22D20050433C
S31508007310AF2292008018814216D300202049C86007
S31508007320084600E011E034308079012803D10621AF
S315080073301C48017502E000211A4801750121C9039C
S315080073400920C006FBF739FE1BE0164840790028DD
S3150800735016D11348C0681A49884211D9FCF778FF34
S3150800736000200F49C8600F487C384088032803DA94
S3150800737001210C48017503E000210A4801750171D5
S3150800738000BF00BF06484068FF21F531884202D990
S315080073900020034948607E20FDF7E4FA00BF3DE679
S315080073A0CC0100208C030020C4000020B80B00008C
S315080073B000040048777269746500000030750000A3
S315080073C010270000F8B5054600247D21C900284687
S315080073D0FAF7A0FA064600270020009000BF0BE047
S315080073E0A1000C48405AB04205DCA100094808181B
S315080073F0408800900127641C06480E380089A04280
S31508007400EEDC002F03D103480E38008A009000985E
S31508007410F8BD00001E02002000C1814001C0804165
S3150800742001C0804100C1814001C0804100C1814046
S3150800743000C1814001C0804101C0804100C1814036
S3150800744000C1814001C0804100C1814001C0804126
S3150800745001C0804100C1814001C0804100C1814016
S3150800746000C1814001C0804100C1814001C0804106
S3150800747001C0804100C1814000C1814001C08041F6
S3150800748001C0804100C1814001C0804100C18140E6
S3150800749000C1814001C0804101C0804100C18140D6
S315080074A000C1814001C0804100C1814001C08041C6
S315080074B001C0804100C1814000C1814001C08041B6
S315080074C001C0804100C1814001C0804100C18140A6
S315080074D000C1814001C0804100C1814001C0804196
S315080074E001C0804100C1814001C0804100C1814086
S315080074F000C1814001C0804101C0804100C1814076
S3150800750000C1814001C0804100C1814001C0804165
S3150800751001C0804100C1814000C0C101C30302C24D
S31508007520C60607C705C5C404CC0C0DCD0FCFCE0EB5
S315080075300ACACB0BC90908C8D81819D91BDBDA1A25
S315080075401EDEDF1FDD1D1CDC14D4D515D71716D695
S31508007550D21213D311D1D010F03031F133F3F23205
S3150800756036F6F737F53534F43CFCFD3DFF3F3EFE75
S31508007570FA3A3BFB39F9F83828E8E929EB2B2AEAE5
S31508007580EE2E2FEF2DEDEC2CE42425E527E7E62655
S3150800759022E2E323E12120E0A06061A163A3A262C5
S315080075A066A6A767A56564A46CACAD6DAF6F6EAE35
S315080075B0AA6A6BAB69A9A86878B8B979BB7B7ABAA5
S315080075C0BE7E7FBF7DBDBC7CB47475B577B7B67615
S315080075D072B2B373B17170B0509091519353529285
S315080075E096565797559594549C5C5D9D5F9F9E5EF5
S315080075F05A9A9B5B99595898884849894B8B8A4A65
S315080076004E8E8F4F8D4D4C8C4484854587474686D4
S31508007610824243834181804038760008C8000020B2
S3150800762004010000E84A00083C770008CC01002065
S315080076303C080000F84A00080000000000000000AE
S31508007640000000000000000000000000000000002C
S31508007650000000000000000000000000000000001C
S31508007660000000000000000000000000000000000C
S3150800767001020304010203040607080900A24A04DA
S3150800768000000000000000000102030406070809C4
S3150800769000000000000000000000000000000000DC
S315080076A000000000040000000100000000000000C7
S315080076B000000000000000000000000000000000BC
S315080076C000000000000000000000000000000000AC
S315080076D0000000000000000000000000000000009C
S315080076E000000000000000000000011058594C4C32
S315080076F0303131327878787878787878CB7E0001AE
S315080077001058594C4C303131327878787878787806
S315080077107804013205054C4C303131061459413292
S3150800772030303532384834353034324178787878E4
S31108007730787D5D7E00000000000000006F
S705080018C515
